:100000009F010F3083169F00FF308600BF308700AE
:1000100005308312A3008316871707179801181756
:100020009816181583129801981718171816981112
:100030000130831699008312A701A401EF106F10FD
:100040008C1E202818186F141A08A5006F1C34285D
:1000500023082502031D312898115A30A600EF14F9
:1000600032289815A701792800308A002708393EE0
:1000700082003A2800308A00250EA800A80C280C1F
:100080000339433E820079287928792847280030AF
:100090008A00250CA800A80C280C0739503E8200C5
:1000A0007928792879287928792879287928582869
:1000B00000308A00073025055E3E820079287928C5
:1000C0007928792866286728722876287928EF14F5
:1000D000A601163024020318712824087F20A600E8
:1000E000A40A7928A401A601EF147928A601EF1427
:1000F0009815EF1C7E282608C720A8201E288400FB
:1001000000308A000408853E820010340034053433
:10011000013403340834533468346134663474343D
:1001200032342D34413407344734723461346D3401
:1001300073346F346E34FF30A900FF30AA008C1E78
:10014000A3281A080800AA0B9F28A90B9D28FC3495
:100150008C1EA8281A080800A000200E0F39B42011
:100160000F302005B4200034A1000A30210203180A
:100170003730031C3030A1072108C720003420305D
:10018000C72000340D30C7200A30C7200034A20039
:0A0190000C1EC82822089900003454
:02400E000A3E68
:02401000BC3FB3
:00000001FF
